S01E000062696E2F64656D6F70726F675F73746D33326C3437362E737265631C
S31508002800008001203D2E00088D2E00088D2E000820
S315080028108D2E00088D2E00088D2E00080000000061
S315080028200000000000000000000000008D2E0008D7
S315080028308D2E0008000000008D2E00081D330008AC
S315080028408D2E00088D2E00088D2E00088D2E00086E
S315080028508D2E00088D2E00088D2E00088D2E00085E
S315080028608D2E00088D2E00088D2E00088D2E00084E
S315080028708D2E00088D2E00088D2E00088D2E00083E
S315080028808D2E00088D2E00088D2E00088D2E00082E
S315080028908D2E00088D2E00088D2E00088D2E00081E
S315080028A08D2E00088D2E00088D2E00088D2E00080E
S315080028B08D2E00088D2E00088D2E00088D2E0008FE
S315080028C08D2E00088D2E00088D2E00088D2E0008EE
S315080028D08D2E00088D2E00088D2E00088D2E0008DE
S315080028E08D2E00088D2E00088D2E00088D2E0008CE
S315080028F08D2E00088D2E00088D2E00088D2E0008BE
S315080029008D2E00088D2E00088D2E00088D2E0008AD
S315080029108D2E00088D2E00088D2E00088D2E00089D
S315080029208D2E00088D2E00088D2E00088D2E00088D
S315080029308D2E00088D2E00088D2E00088D2E00087D
S315080029408D2E00088D2E00088D2E00088D2E00086D
S315080029508D2E00088D2E00088D2E00088D2E00085D
S315080029608D2E00088D2E00088D2E00088D2E00084D
S315080029708D2E00088D2E00088D2E00080000000000
S311080029808D2E00088D2E0008EE11AA55B9
S3150800298C10B5054C237833B9044B13B10448AFF38F
S3150800299C00800123237010BD2C04002000000000C9
S315080029AC904B0008084B10B51BB108490848AFF303
S315080029BC00800848036803B910BD074B002BFBD0F1
S315080029CCBDE81040184700BF000000003004002086
S315080029DC904B00082C0400200000000053B94AB99B
S315080029EC002908BF00281CBF4FF0FF314FF0FF30FD
S315080029FC00F07EB9ADF1080C6DE904CE00F006F8CE
S31508002A0CDDF804E0DDE9022304B070472DE9F04750
S31508002A1C8C460E460446089D002B50D18A42174612
S31508002A2C6CD9B2FA82FEBEF1000F0BD0CEF120049F
S31508002A3C20FA04F401FA0EF644EA060C02FA0EF72A
S31508002A4C00FA0EF44FEA1749220CBCFBF9F01FFAF0
S31508002A5C87F809FB10C642EA064600FB08F3B342A0
S31508002A6C09D9F61900F1FF3280F02281B34240F2FF
S31508002A7C1F8102383E44F61AA2B2B6FBF9F309FBDB
S31508002A8C136642EA064403FB08F8A04509D9E4197B
S31508002A9C03F1FF3280F00A81A04540F20781023B20
S31508002AAC3C44C8EB040443EA00400021002D62D0E4
S31508002ABC24FA0EF400232C606B60BDE8F0878B4279
S31508002ACC07D9002D55D0002185E841000846BDE8F8
S31508002ADCF087B3FA83F1002940F09080B34202D311
S31508002AEC824200F2F880841A66EB03060120B4468B
S31508002AFC002D40D085E81010BDE8F08712B90127E3
S31508002B0CB7FBF2F7B7FA87FEBEF1000F35D1F31B08
S31508002B1C4FEA17481FFA87FC0121B3FBF8F0220C81
S31508002B2C08FB103642EA06460CFB00F3B34207D9FB
S31508002B3CF61900F1FF3202D2B34200F2CE801046EB
S31508002B4CF61AA2B2B6FBF8F308FB136642EA064479
S31508002B5C0CFB03FCA44507D9E41903F1FF3202D296
S31508002B6CA44500F2B5801346CCEB040443EA0040B6
S31508002B7C9CE729462846BDE8F087CEF1200106FADF
S31508002B8C0EF307FA0EF720FA01F94FEA1748CE406A
S31508002B9C49EA0309B6FBF8FA4FEA194408FB1A6620
S31508002BAC1FFA87FC44EA06430AFB0CF29A4200FA1F
S31508002BBC0EF40AD9DB190AF1FF3180F087809A42A4
S31508002BCC40F28480AAF1020A3B449B1A1FFA89F93F
S31508002BDCB3FBF8F108FB113349EA034301FB0CF686
S31508002BEC9E4207D9DB1901F1FF326BD29E4269D995
S31508002BFC02393B449B1B41EA0A418EE7C1F1200E80
S31508002C0C22FA0EF48B40234320FA0EF706FA01F447
S31508002C1C4FEA134C26FA0EF63C43B6FBFCF9270C86
S31508002C2C0CFB19661FFA83F847EA064609FB08F7F0
S31508002C3CB74202FA01F200FA01FA08D9F61809F1B4
S31508002C4CFF3041D2B7423FD9A9F102091E44F61BFF
S31508002C5CA0B2B6FBFCF40CFB146640EA064704FB70
S31508002C6C08F8B84507D9FF1804F1FF3028D2B8453B
S31508002C7C26D9023C1F4444EA0940C8EB0707A0FBC7
S31508002C8C02894F4544464E4614D329D065B3BAEB50
S31508002C9C040367EB060707FA0EFECB40CF404EEA55
S31508002CAC030385E888000021BDE8F0871346F8E69B
S31508002CBC1046E0E6B8EB020469EB03060138E5E7D3
S31508002CCC0446D8E7114695E78146C0E78A467CE76D
S31508002CDC023B3C4448E708460AE702383E442FE7DD
S31508002CECC245E7D33E46D1E72946BDE8F08700BF83
S31508002CFC704700BF70B50F4E0F4D761BB61018BF38
S31508002D0C002405D0013455F8043B9847A642F9D15E
S31508002D1C0A4E0B4D761B01F035FFB61018BF002472
S31508002D2C06D0013455F8043B9847A642F9D170BD34
S31508002D3C70BD00BF204C0008204C0008284C000829
S31508002D4C204C0008024B13B1024800F005B8704736
S31508002D5C00000000712D0008002301461A4618468B
S31508002D6C00F014B838B5074D074C2C1BA41005D029
S31508002D7C013C55F8043D9847002CF9D1BDE838407C
S31508002D8C01F006BF2C4C0008284C00082DE9F0472A
S31508002D9C254C2568D5F848410646884692469946F4
S31508002DACC4B360681F2817DC431C76B104EB800596
S31508002DBC0122C5F888A0D4F8881182401143022E46
S31508002DCCC4F88811C5F808911ED00230636044F81F
S31508002DDC20800020BDE8F087144B03B34FF4C8706D
S31508002DECAFF300800446D0B1D5F84831002780E807
S31508002DFC8800C5F8484138460123C4F88871C4F8D8
S31508002E0C8C71002EE1D0D1E7D4F88C110A43C4F8A2
S31508002E1C8C21DAE705F5A674C5F84841C1E74FF0E9
S31508002E2CFF30BDE8F08700BFA84B00080000000083
S31508002E3CDFF834D0002103E00C4B5B5843500431C7
S31508002E4C0B480C4B42189A42F6D30B4A02E0002365
S31508002E5C42F8043B094B9A42F9D300F05FFAFFF7A4
S31508002E6C49FF00F071F9FEE7008001202C4C0008A0
S31508002E7C000000202C0400202C0400203C05002017
S31508002E8CFEE70000F0B59C46002420E0124D15F82C
S31508002E9C147005EB440595F801E007EB0E0505FBE8
S31508002EAC00050E4B93FBF5F605FB16366EB993FB30
S31508002EBCF5F5ADB20D80013DADB2B5F5806F04D216
S31508002ECC17708CF800E00120F0BD0134E4B2112C27
S31508002EDCDCD90020F0BD00BFAC4B000880380100DF
S31508002EEC08B50948094B03604FF461434360002356
S31508002EFC8360C360036183610C224261C361036210
S31508002F0C436201F0B3FA08BD4804002000440040AF
S31508002F1C30B58DB000258DF82D500CAB03F8045D3B
S31508002F2C0DF12D020DF12E014FF4FA70FFF7AAFFE1
S31508002F3C1A4C1B4B236025766576A576E5762577A0
S31508002F4C6577A560E5609DF82D30013B1B04236170
S31508002F5C9DF82C30013B1B056361BDF82E30636070
S31508002F6C204601F017FC06950795012308934CF6A5
S31508002F7CE042019202954FF6E07203920422049203
S31508002F8C059509930E230A930DEB0201204601F0D1
S31508002F9CABFC204601F026FD0DB030BDC404002064
S31508002FAC0064004008B5002301220146034801F0DD
S31508002FBC9FF908B9012008BD002008BD4804002067
S31508002FCC08B5FFF78DFFFFF7A3FF08BDBFF34F8FBB
S31508002FDC0549CA6802F4E062044B1343CB60BFF39D
S31508002FEC4F8F00BFFDE700BF00ED00E00400FA05B7
S31508002FFC08B5204B1B789BB91F48FFF7D3FF012850
S3150800300C36D11D4B1B78002B32D000F07DF91B4BAB
S3150800301C18600122174B1A700022194B1A7008BD3A
S3150800302C174B1B78013314481844FFF7BBFF0128CC
S3150800303C14D1134A13780133DBB213700E4A127883
S3150800304C934215D100220B4B1A700B4B5B78FF2B56
S3150800305C0ED1094B9B785BB9FFF7B8FF00F054F912
S3150800306C064B1B686433984202D90022014B1A702E
S3150800307C08BD00BF2E050020EC040020C00400206B
S3150800308C2D05002000B58BB001AB03AA00210E4814
S3150800309C01F0D8FCA8B940F26763039A9A4203D1A7
S315080030AC059B1BB1002302E0002300E0012343B17A
S315080030BC9DF80430FF2B04D19DF805300BB9FFF7AA
S315080030CC85FF0BB05DF804FBC404002008B5FFF7B8
S315080030DC8FFFFFF7D7FF08BD00B597B002230593FE
S315080030EC4FF480720892102209920F9310930122C2
S315080030FC11920A221292072213921493159305A879
S3150800310C00F0FAF900B1FEE70F23009303210191B1
S3150800311C0023029303930493684600F0B9FC00B1AC
S3150800312CFEE74FF4007000F0C1FD00B1FEE717B0E2
S3150800313C5DF804FB08B500F017FEFFF7CDFF00F0AD
S3150800314CCDF800F09DF808BD08B5FFF7F3FFFFF7BB
S3150800315C37FF00F09DF8FFF7B9FFFAE770B58CB0AA
S3150800316C454B1A6E42F001021A661A6E02F00102FB
S3150800317C0192019A9A6D42F080529A659A6D02F004
S3150800318C80520292029ADA6C42F00102DA64DA6C24
S3150800319C02F001020392039ADA6C42F00202DA6434
S315080031ACDA6C02F002020492049A9A6D42F4003226
S315080031BC9A659A6D02F400320592059A9A6D42F058
S315080031CC00729A659B6D03F000730693069B0320A9
S315080031DC01F06EFA002211466FF00B0001F07AFA34
S315080031EC002211466FF00A0001F074FA002211460B
S315080031FC6FF0090001F06EFA002211466FF0040018
S3150800320C01F068FA002211466FF0030001F062FA29
S3150800321C002211466FF0010001F05CFA00221146FB
S3150800322C4FF0FF3001F056FA202307930123089339
S3150800323C002409940A9407A94FF0904001F04CF920
S3150800324C0C23079302260896099403250A95072347
S3150800325C0B9307A94FF0904001F03EF94FF44073D9
S3150800326C0793089609940A9509230B9307A903480B
S3150800327C01F032F90CB070BD001002400004004891
S3150800328C08B5002220214FF0904001F00BFA08BD3A
S3150800329C10B500F039F80F4B1B68C31AB3F5FA7F53
S315080032AC16D304460C4B1B7843B901220A4B1A70E9
S315080032BC20214FF0904001F0F5F907E00022064B6B
S315080032CC1A7020214FF0904001F0ECF9014B1C606C
S315080032DC10BD00BF300500203405002008B500F0ED
S315080032ECB7FC084BA3FB0030800901F025FA042033
S315080032FC01F038FA002211464FF0FF3001F0EAF9D6
S3150800330C08BD00BFD34D621008B500F047FD08BDD7
S3150800331C08B500F03BFD01F037FA08BD0F49D1F8A6
S3150800332C883043F47003C1F888300D4B1A6842F0A4
S3150800333C01021A60002098601A6822F0A85222F43A
S3150800334C10221A604FF48052DA601A6822F480222E
S3150800335C1A609861034B8B60704700BF00ED00E064
S3150800336C001002400028000830B583B00546204BF3
S3150800337C9B6D13F0805F02D000F090FC0FE01C4CA4
S3150800338CA36D43F08053A365A36D03F0805301939B
S3150800339C019B00F083FCA36D23F08053A365B0F565
S315080033AC007F05D1802D0AD9A02D0AD902210FE05C
S315080033BC802D08D809D0702D09D0002108E00021ED
S315080033CC06E0012104E0032102E0022100E00121CC
S315080033DC084A136823F007030B431360136803F0BA
S315080033EC0703994201D0012000E0002003B030BD4C
S315080033FC00100240002002403B4B9B6813F00C0F58
S3150800340C0BD0394B9B6803F00C030C2B1ED1364B97
S3150800341CDB6803F00303012B18D1334B1B6813F03D
S3150800342C080F05D1304BD3F89430C3F3032303E0CC
S3150800343C2D4B1B68C3F303132C4A52F823102A4B43
S3150800344C9B6813F00C0F10D0002015E0264B9B68D8
S3150800345C03F00C03042B0AD0234B9B6803F00C03D4
S3150800346C082B07D00020014606E0084604E0204851
S3150800347C002101E01F4800211B4A926802F00C0249
S3150800348C0C2A30D1184BDA6802F00302DB68C3F356
S3150800349C02130133022A02D0032A0AD013E0144875
S315080034ACB0FBF3F0104BDB68C3F3062303FB00F306
S315080034BC11E01048B0FBF3F30B4AD268C2F30622AC
S315080034CC02FB03F307E0B1FBF3F3074AD268C2F336
S315080034DC062202FB03F3044AD068C0F341600130AC
S315080034EC4000B3FBF0F0704700100240E84B0008B0
S315080034FC0024F40000127A0070B582B00446036802
S3150800350C13F0100F00F09D80A74B9B6813F00C0F5F
S3150800351C5AD1A54B1B6813F0020F03D08369002BF5
S3150800352C00F08782206AA04B1B6813F0080F04D0A2
S3150800353C9D4B1B6803F0F00305E09B4BD3F89430C6
S3150800354C1B0903F0F003834217D2FFF70DFF00287F
S3150800355C40F07182944B1A6842F008021A601A6895
S3150800356C22F0F001226A0A431A605A6822F47F4252
S3150800357CE16942EA01225A6017E08B4B1A6842F05D
S3150800358C08021A601A6822F0F001226A0A431A60C5
S3150800359C5A6822F47F42E16942EA01225A60206A9B
S315080035ACFFF7E2FE002840F04882FFF725FF7E4B26
S315080035BC9B68C3F303137D4AD35CD8407C4B1860D5
S315080035CC002000F0BBFB3CE0836933B3764A1368F2
S315080035DC43F00103136000F0E1FB054605E000F03B
S315080035ECDDFB401B022800F22A826F4B1B6813F086
S315080035FC020FF4D06C4B1A6842F008021A601A686B
S3150800360C22F0F001226A0A431A605A6822F47F42B1
S3150800361CE16942EA01225A6013E0634A136823F00F
S3150800362C0103136000F0BAFB054605E000F0B6FB93
S3150800363C401B022800F205825B4B1B6813F0020F35
S3150800364CF4D1236813F0010F5ED0574B9B6803F037
S3150800365C0C03082B0BD0544B9B6803F00C030C2B58
S3150800366C0ED1514BDB6803F00303032B08D14E4BE9
S3150800367C1B6813F4003F47D06368002B44D1E2E182
S3150800368C6368B3F5803F05D1474A136843F4803322
S3150800369C136018E0B3F5A02F0CD103F18043A3F502
S315080036AC3C331A6842F480221A601A6842F4803253
S315080036BC1A6008E03C4B1A6822F480321A601A68C1
S315080036CC22F480221A6063687BB100F067FB05461A
S315080036DC05E000F063FB401B642800F2B681324B10
S315080036EC1B6813F4003FF4D00EE000F057FB0546B8
S315080036FC05E000F053FB401B642800F2A8812A4B16
S3150800370C1B6813F4003FF4D1236813F0020F5CD046
S3150800371C254B9B6803F00C03042B0BD0224B9B68A0
S3150800372C03F00C030C2B17D11F4BDB6803F00303B8
S3150800373C022B11D11C4B1B6813F4806F03D0E36862
S3150800374C002B00F08681184A536823F0F853216938
S3150800375C43EA0163536038E0E368E3B1124A13683D
S3150800376C43F48073136000F019FB054605E000F07E
S3150800377C15FB401B022800F26E810B4B1B6813F4D9
S3150800378C806FF4D0084A536823F0F853216943EA4A
S3150800379C0163536019E0044A136823F480731360B9
S315080037AC00F0FCFA05460BE000100240D04B00086E
S315080037BC2804002000F0F2FA401B022800F24D8182
S315080037CCB14B1B6813F4806FF4D1236813F0080F00
S315080037DC30D06369BBB1AC4AD2F8943043F00103DC
S315080037ECC2F8943000F0DAFA054605E000F0D6FA8D
S315080037FC401B022800F23381A34BD3F8943013F004
S3150800380C020FF3D016E0A04AD2F8943023F0010345
S3150800381CC2F8943000F0C2FA054605E000F0BEFA8C
S3150800382C401B022800F21D81974BD3F8943013F0F5
S3150800383C020FF3D1236813F0040F7FD0924B9B6DC4
S3150800384C13F0805F0BD1904B9A6D42F080529A65BB
S3150800385C9B6D03F080530193019B012500E0002525
S3150800386C8A4B1B6813F4807F13D1884A136843F478
S3150800387C8073136000F092FA064605E000F08EFAA3
S3150800388C801B022800F2EF80804B1B6813F4807FA4
S3150800389CF4D0A368012B07D17B4AD2F8903043F0B9
S315080038AC0103C2F890301CE0052B0DD1764BD3F8EA
S315080038BC902042F00402C3F89020D3F8902042F0EE
S315080038CC0102C3F890200CE06F4BD3F8902022F03D
S315080038DC0102C3F89020D3F8902022F00402C3F812
S315080038EC9020A36893B100F059FA064607E000F059
S315080038FC55FA801B41F28833984200F2B680624B27
S3150800390CD3F8903013F0020FF1D011E000F046FA1C
S3150800391C064607E000F042FA801B41F288339842CB
S3150800392C00F2A580584BD3F8903013F0020FF1D162
S3150800393C25B1554A936D23F080539365A36A002BE2
S3150800394C00F09780504A926802F00C020C2A00F09C
S3150800395C9280022B43D14C4A136823F08073136070
S3150800396C00F01CFA054605E000F018FA401B022880
S3150800397C00F28380444B1B6813F0007FF4D1236B51
S3150800398C5A1E636B1B0243EA0213A26B120943EA23
S3150800399C4242E36A1343E26B5208013A43EA425342
S315080039AC226C5208013A43EA4263374AD3601368D9
S315080039BC43F080731360D36843F08073D36000F0D0
S315080039CCEDF9044604E000F0E9F9001B022856D884
S315080039DC2D4B1B6813F0007FF5D0002052E02A4BC4
S315080039EC1A6822F080721A601B6813F0006F09D1EE
S315080039FC254B1B6813F0005F04D1234AD36823F0C8
S31508003A0C0303D360204AD36823F0887323F48033E6
S31508003A1CD36000F0C3F9044604E000F0BFF9001BBC
S31508003A2C02282ED8184B1B6813F0007FF5D10020FE
S31508003A3C28E0012026E0012024E0012022E00320D2
S31508003A4C20E003201EE001201CE003201AE00320DE
S31508003A5C18E0012016E0032014E0032012E00320EE
S31508003A6C10E003200EE003200CE003200AE00320FC
S31508003A7C08E0002006E0012004E0032002E0032011
S31508003A8C00E0032002B070BD001002400070004038
S31508003A9C70B56B4B1B6803F007038B420BD2684A55
S31508003AAC136823F007030B431360136803F007032B
S31508003ABC994240F0B0800D460446036813F0010F96
S31508003ACC66D04368032B05D15E4A126812F0007F54
S31508003ADC15D1A2E0022B05D15A4A126812F4003FFE
S31508003AEC0DD19CE02BB9574A126812F0020F06D179
S31508003AFC97E0544A126812F4806F00F0948051498A
S31508003B0C8A6822F0030213438B6000F047F90646D5
S31508003B1C6368032B0FD107E000F040F9801B41F2D4
S31508003B2C8833984200F28180464B9B6803F00C035D
S31508003B3C0C2BF1D12CE0022B0ED106E000F02EF95D
S31508003B4C801B41F28833984271D83E4B9B6803F030
S31508003B5C0C03082BF2D11BE03BB113E000F01EF965
S31508003B6C801B41F28833984263D8364B9B6813F016
S31508003B7C0C0FF3D10CE000F011F9801B41F28833DD
S31508003B8C984258D82F4B9B6803F00C03042BF2D1A0
S31508003B9C236813F0020F06D02A498B6823F0F0022B
S31508003BACA36813438B60264B1B6803F007039D42DF
S31508003BBC0AD2234A136823F007032B4313601368AE
S31508003BCC03F007039D4238D1236813F0040F06D07F
S31508003BDC1C498B6823F4E062E36813438B60236803
S31508003BEC13F0080F07D0174A936823F4605321691A
S31508003BFC43EAC1039360FFF7FFFB124B9B68C3F3C1
S31508003C0C0313114AD35CD840104B1860002000F0FF
S31508003C1C95F8002070BD012070BD012070BD0120F3
S31508003C2C70BD012070BD012070BD032070BD03203E
S31508003C3C70BD032070BD032070BD012070BD00BF90
S31508003C4C0020024000100240D04B00082804002037
S31508003C5C014B1868704700BF2804002008B5FFF709
S31508003C6CF7FF044B9B68C3F30223034AD35CD84083
S31508003C7C08BD00BF00100240E04B000808B5FFF76E
S31508003C8CE7FF044B9B68C3F3C223034AD35CD840B3
S31508003C9C08BD00BF00100240E04B0008024B186834
S31508003CAC00F4C060704700BF00700040B0F5007F9C
S31508003CBC2AD1204B1B6803F4C063B3F5007F33D0BD
S31508003CCC1C4A136823F4C06343F4007313601A4B3D
S31508003CDC1B6802F1467202F55B3202F28322A2FBE2
S31508003CEC03239A0C322303FB02F300E0013B23B1B6
S31508003CFC104A526912F4806FF8D10E4B5B6913F4B3
S31508003D0C806F13D0032070470A4B1B6803F4C063FB
S31508003D1CB3F5806F0CD0074A136823F4C06343F4D9
S31508003D2C806313600020704700207047002070479E
S31508003D3C00207047007000402804002010B5044687
S31508003D4C074B1B680748A0FB0330800900F0F4FCFE
S31508003D5C002221464FF0FF3000F0BCFC002010BDBD
S31508003D6C28040020D34D621008B5074A136843F49B
S31508003D7C80731360032000F09BFC0020FFF7DEFF26
S31508003D8CFFF7ECF9002008BD00200240024A136830
S31508003D9C01331360704700BF38050020014B1868C3
S31508003DAC704700BF38050020704700BF2DE9784BD7
S31508003DBC0446826803691A4343691A43C3691A435A
S31508003DCC01680868A04B034013430B6021684B68D5
S31508003DDC23F44052E36813434B60A16922689B4B5A
S31508003DEC9A4201D0236A1943936823F430630B4330
S31508003DFC93602368964A934213D102F55842D2F837
S31508003E0C882002F00302032A09D8DFE802F002042C
S31508003E1C98060125A0E004259EE008259CE01025BF
S31508003E2C9AE08C4A934218D102F5E632D2F88820E9
S31508003E3C02F00C020C2A0ED8DFE802F0070D0D0D65
S31508003E4C090D0D0D830D0D0D0B00002584E00425C1
S31508003E5C82E0082580E010257EE07F4A934217D140
S31508003E6C02F5E432D2F8882002F03002102A09D082
S31508003E7C01D82AB10AE0202A65D0302A04D005E0F8
S31508003E8C002569E0042567E0082565E0102563E050
S31508003E9C724A934217D102F5E232D2F8882002F020
S31508003EACC002402A09D001D82AB10AE0802A4CD08F
S31508003EBCC02A04D005E000254EE004254CE0082570
S31508003ECC4AE0102548E0664A93421AD102F5E032D8
S31508003EDCD2F8882002F44072B2F5807F0BD001D854
S31508003EEC3AB10CE0B2F5007F31D0B2F5407F04D080
S31508003EFC05E0002530E004252EE008252CE01025E9
S31508003F0C2AE0524A934224D102F5C832D2F88820C4
S31508003F1C02F44062B2F5806F0BD001D83AB10CE0CE
S31508003F2CB2F5006F17D0B2F5406F04D005E0002546
S31508003F3C12E0042510E008250EE010250CE00225F9
S31508003F4C0AE0022508E0022506E0022504E002251F
S31508003F5C02E0102500E002253C4A934240F0888096
S31508003F6C082D11D8DFE805F0081005100C101010F4
S31508003F7C13003C4800260DE0FFF770FE002609E00A
S31508003F8CFFF73AFA002605E00020012602E04FF476
S31508003F9C00400026002800F00C81626802EB420300
S31508003FAC9842C0F0FD80B0EB023F00F2FB80082D72
S31508003FBC3ED8DFE805F0053D173D213D3D3D330074
S31508003FCCFFF74CFE00234FEA10694FEA0028626897
S31508003FDC500818EB000B49F1000C58466146FEF7E1
S31508003FECFDFC27E0550800231F480021401941F124
S31508003FFC0001FEF7F3FC1DE0FFF7FEF900234FEA7C
S3150800400C10694FEA00286268500818EB000B49F152
S3150800401C000C58466146FEF7E1FC0BE050080021FF
S3150800402C002310F5000041F10001FEF7D7FC01E072
S3150800403C01260020A0F540720C4B9A4200F2B4807F
S3150800404C2368D860B5E000BFF369FFEF0080004035
S3150800405C003801400044004000480040004C004035
S3150800406C005000400024F400000024F4FFFC0F006C
S3150800407CE369B3F5004F4DD1082D3BD8DFE805F0C1
S3150800408C05101B3A263A3A3A3100FFF7E7FD636802
S3150800409C5A0802EB4000B0FBF3F39BB200262BE068
S315080040ACFFF7ECFD63685A0802EB4000B0FBF3F32C
S315080040BC9BB2002620E061684A0802F1F47303F506
S315080040CC9043B3FBF1F39BB2002615E0FFF794F986
S315080040DC63685A0802EB4000B0FBF3F39BB2002668
S315080040EC0AE06268530803F58033B3FBF2F39BB21C
S315080040FC002601E001260023A3F110014FF6EF720A
S3150800410C914253D823F00F02C3F342031343226898
S3150800411CD3604EE0082D38D8DFE805F0050F1937BF
S3150800412C243737372E00FFF799FD636800EB5300E9
S3150800413CB0FBF3F080B2002629E0FFF79FFD636819
S3150800414C00EB5300B0FBF3F080B200261FE060686A
S3150800415C420802F5740303F51053B3FBF0F080B272
S3150800416C002614E0FFF748F9636800EB5300B0FB30
S3150800417CF3F080B200260AE06068430803F50043B2
S3150800418CB3FBF0F080B2002601E001260020A0F176
S3150800419C10024FF6EF739A420AD82368D86008E0E3
S315080041AC012606E0012604E0012602E0012600E0CD
S315080041BC01260023236663663046BDE8788B00BF6C
S315080041CC436A13F0010F06D001684B6823F40032DA
S315080041DC836A13434B60436A13F0020F06D00168D7
S315080041EC4B6823F48032C36A13434B60436A13F05B
S315080041FC040F06D001684B6823F48022036B134323
S3150800420C4B60436A13F0080F06D001684B6823F419
S3150800421C0042436B13434B60436A13F0100F06D0EE
S3150800422C01688B6823F48052836B13438B60436A53
S3150800423C13F0200F06D001688B6823F40052C36B69
S3150800424C13438B60436A13F0400F11D001684B6817
S3150800425C23F48012036C13434B60036CB3F5801F75
S3150800426C06D101684B6823F4C002436C13434B60B8
S3150800427C436A13F0800F06D001684B6823F40022BA
S3150800428C836C13434B6070472DE9F04105460F4686
S3150800429C16469846069C1EE0B4F1FF3F1BD02CB17F
S315080042ACFFF77CFDC8EB0000844214D22A68136819
S315080042BC23F4D07313602A68936823F00103936080
S315080042CC202385F8713085F87230002385F8703014
S315080042DC0320BDE8F0812B68DB6937EA03030CBFC2
S315080042EC01230023B342D7D00020BDE8F08100BFDC
S315080042FC2DE9F04182B01E4690F87230DBB2202BC5
S3150800430C71D104460D46904600296ED0002A6ED00F
S3150800431C90F87030012B6CD0012380F87030002394
S3150800432C4367222380F87230FFF738FD0746A4F856
S3150800433C5880A4F85A80A368B3F5805F0AD123691C
S3150800434C23B940F2FF13A4F85C301AE0FF23A4F853
S3150800435C5C3016E04BB923691BB9FF23A4F85C3013
S3150800436C0FE07F23A4F85C300BE0B3F1805F08D133
S3150800437C23691BB97F23A4F85C3002E03F23A4F819
S3150800438C5C30B4F85C8022E000963B460022202183
S3150800439C2046FFF779FF70BBA368B3F5805F08D199
S315080043AC236933B923689B8C08EA030325F8023B77
S315080043BC06E023689B8C5FFA88F213402B70013554
S315080043CCB4F85A309BB2013B9BB2A4F85A30B4F8F5
S315080043DC5A309BB2002BD7D1202384F87230002098
S315080043EC84F8700008E0022006E0012004E00120B1
S315080043FC02E0022000E0032002B0BDE8F08100BF15
S3150800440C30B583B0044600234367FFF7C7FC05465F
S3150800441C23681B6813F0080F0AD06FF07E430093CD
S3150800442C034600224FF400112046FFF72DFFC0B9B2
S3150800443C23681B6813F0040F0AD06FF07E430093B1
S3150800444C2B4600224FF480012046FFF71DFF50B97A
S3150800445C202384F8713084F87230002084F87000B8
S3150800446C02E0032000E0032003B030BD80B310B592
S3150800447C044690F8713013F0FF0F04D1002380F82E
S3150800448C7030FFF791FC242384F871302268136886
S3150800449C23F0010313602046FFF788FC012819D086
S315080044AC636A13B12046FFF78BFE2268536823F420
S315080044BC904353602268936823F02A03936022681A
S315080044CC136843F0010313602046FFF799FF10BDEC
S315080044DC0120704710BD00BFF0B583B00023D1E0B2
S315080044EC01249C40224000F0CC804D68022D01D05E
S315080044FC122D10D1DE08083650F826C003F0070531
S3150800450CAF000F25BD402CEA050E0D69BD404EEADD
S3150800451C050540F8265005685F000326BE40F6439D
S3150800452C05EA060E4D6805F00305BD404EEA05057D
S3150800453C05604D6805F1FF3EBEF1010F03D9112D3B
S3150800454C01D0122D11D1856806EA050ECD68BD403D
S3150800455C4EEA05058560456825EA040E4D68C5F3DF
S3150800456C00159D404EEA050545604D6805F0030E9D
S3150800457CBEF1030F08D1D0F82CE02EEA0404C5F3DB
S3150800458CC0059D402C43C462C46826408C68BC4058
S3150800459C3443C4604C6814F0805F72D03D4C256E71
S315080045AC45F001052566246E04F001040194019C6E
S315080045BC9E08B51C384C54F8257003F00304A40067
S315080045CC0F25A54027EA0507B0F1904F18D0334DB3
S315080045DCA84217D005F58065A84215D005F5806563
S315080045ECA84213D005F58065A84211D005F580655B
S315080045FCA8420FD005F58065A8420DD106250CE01A
S3150800460C00250AE0012508E0022506E0032504E05A
S3150800461C042502E0052500E0072505FA04F43C43C9
S3150800462C02361D4D45F826401D4C2568D44305EA2F
S3150800463C04064F6817F4803F01D042EA0506184D68
S3150800464C2E606D6804EA05064F6817F4003F01D022
S3150800465C42EA0506124D6E60AD6804EA05064F6817
S3150800466C17F4801F01D042EA05060D4DAE60ED68C1
S3150800467C2C404E6816F4001F01D042EA0504084A7D
S3150800468CD46001330A6832FA03F47FF429AF03B015
S3150800469CF0BD00BF001002400000014000040048B5
S315080046AC000401400AB1816170478162704700BFFE
S315080046BC074AD36823F4E0631B041B0C000200F4BE
S315080046CCE060184340F0BF6040F40030D06070479B
S315080046DC00ED00E030B4164BDB68C3F30223C3F1DC
S315080046EC0704042C28BF04241D1D062D01D9DD1E24
S315080046FC00E00025012303FA04F4013C2140A940FB
S3150800470CAB40013B1A400A43002806DA00F00F00BA
S3150800471C1201D2B2074B1A5407E01201D2B200F1B9
S3150800472C604000F5614080F8002330BC704700BF3C
S3150800473C00ED00E014ED00E00138B0F1807F0AD2FC
S3150800474C064B5860F021064A82F823100020986020
S3150800475C07221A6070470120704700BF10E000E07E
S3150800476C00ED00E0042805D1054A136843F004035C
S3150800477C13607047024A136823F0040313607047EA
S3150800478C10E000E0704700BF08B5FFF7FBFF08BD57
S3150800479C704700BF002800F0A48038B5044690F88E
S315080047AC203013F0FF0F01D1FFF7F2FF22681368D0
S315080047BC23F002031360FFF7F1FA05460DE0FFF745
S315080047CCEDFA401B0A2808D9636A43F4003363627E
S315080047DC052384F82030012038BD23685A6812F066
S315080047EC020FECD11A6842F001021A60FFF7D6FAEA
S315080047FC05460DE0FFF7D2FA401B0A2808D9636A6A
S3150800480C43F400336362052384F82030012038BD55
S3150800481C23685A6812F0010FECD0227E012A04D1C3
S3150800482C1A6842F080021A6003E01A6822F08002C5
S3150800483C1A60637E012B05D12268136843F0400386
S3150800484C136004E02268136823F040031360A37E08
S3150800485C012B05D12268136843F02003136004E08A
S3150800486C2268136823F020031360E37E012B05D11D
S3150800487C2268136823F01003136004E02268136897
S3150800488C43F010031360237F012B05D122681368AC
S3150800489C43F00803136004E02268136823F0080346
S315080048AC1360637F012B05D12268136843F0040358
S315080048BC136004E02268136823F00403136021686C
S315080048CCA268E3681A4323691A4363691A4363683F
S315080048DC013B1343CB6100206062012384F820302E
S315080048EC38BD0120704700BF70B4036890F82020CB
S315080048FCD2B2012A04D090F82020D2B2022A6AD168
S3150800490CD3F8002242F00102C3F800224A690120BA
S3150800491C00FA02F2D3F81C02D4432040C3F81C0256
S3150800492CC869A8B9D3F80C022040C3F80C02486928
S3150800493CCE688D8845EA0645483043F830504869B4
S3150800494C8E680D8845EA0645483003EBC00045607D
S3150800495CC869012815D1D3F80C021043C3F80C0208
S3150800496C48690E688D8845EA0645483043F8305044
S3150800497C48698E688D8945EA0645483003EBC000C0
S3150800498C4560886928B9D3F804022040C3F80402A4
S3150800499C04E0D3F804021043C3F80402086928B9E2
S315080049ACD3F814020440C3F8144204E0D3F81402F2
S315080049BC1043C3F81402096A012904D1D3F81C124E
S315080049CC0A43C3F81C22D3F8002222F00102C3F8CA
S315080049DC0022002004E0436A43F48023436201204A
S315080049EC70BC704738B590F82030DBB2012B22D159
S315080049FC0446022380F820300268136823F001036A
S31508004A0C1360FFF7CBF905460DE0FFF7C7F9401B16
S31508004A1C0A2808D9636A43F400336362052384F8C9
S31508004A2C2030012038BD23685B6813F0010FECD1E8
S31508004A3C0020606238BD436A43F4002343620120B8
S31508004A4C38BD00BF30B490F82040E4B2012C05D034
S31508004A5C90F82040E4B2022C40F08A8051B90468E0
S31508004A6CE46814F0030F12D1436A43F4001343624B
S31508004A7C012084E001290AD10468246914F0030F83
S31508004A8C05D1436A43F400134362012077E00568B5
S31508004A9C01F11B0424012C5904F0040494603CB95C
S31508004AAC056801F11B0424012C59640D146006E0F9
S31508004ABC056801F11B0424012C59E40854600568A7
S31508004ACC01F11B0424012D59C5F34005D560056871
S31508004ADC25446D6805F00F051561056825446D6854
S31508004AECC5F30725956105682C446468240C546144
S31508004AFC04680A011444D4F8B8411C7004681444B8
S31508004B0CD4F8B841240A5C7004681444D4F8B84143
S31508004B1C240C9C7004681444D4F8B841240EDC7038
S31508004B2C04681444D4F8BC411C7104681444D4F8C1
S31508004B3CBC41240A5C7104681444D4F8BC41240CA6
S31508004B4C9C7104682244D2F8BC21120EDA7131B970
S31508004B5C0268D36843F02003D36000200FE00129D4
S31508004B6C0CD10268136943F020031361002006E098
S31508004B7C436A43F480234362012000E0002030BCE2
S31508004B8C704700BFF8B500BFF8BC08BC9E46704716
S31108004B9CF8B500BFF8BC08BC9E46704780
S31508004BA80000002005020602060307030803090396
S31508004BB809040A040B040C040C050D050E050F055B
S31508004BC80F06100610071008000000000000000075
S31508004BD8010203040607080900000000010203048D
S31508004BE8A0860100400D0300801A060000350C0057
S31508004BF840420F0080841E0000093D0000127A001A
S31508004C080024F40000366E010048E801006CDC0256
S30D08004C1800DEFF7F0100000029
S30D08004C20512D0008B129000816
S30908004C288D290008BC
S31508004C2C00000000EC02002054030020BC03002006
S31508004C3C000000000000000000000000000000005A
S31508004C4C000000000000000000000000000000004A
S31508004C5C000000000000000000000000000000003A
S31508004C6C000000000000000000000000000000002A
S31508004C7C000000000000000000000000000000001A
S31508004C8C000000000000000000000000000000000A
S31508004C9C00000000000000000000000000000000FA
S31508004CAC00000000000000000000000000000000EA
S31508004CBC00000000000000000000000000000000DA
S31508004CCC00000000000000000100000000000000C9
S31508004CDC0E33CDAB34126DE6ECDE05000B0000008E
S31508004CEC00000000000000000000000000000000AA
S31508004CFC000000000000000000000000000000009A
S31508004D0C0000000000000000000000000000000089
S31508004D1C0000000000000000000000000000000079
S3110800504C000000000000000000093D0004
S70508002E3D87
